:10000000E3EF03F01200FFFF04EF04F01200FFFF24
:100018000CEF04F01200FFFFFFFFFFFFFFFFFFFFE1
:10002A000100DE0700007E0000000200000000015F
:10003A00776B1E0E716E0401400E096F200E0A6F57
:10004A00040E0B6F880E086F0401200E0E6F040E4B
:10005A000F6F400E0C6F1200550EA76EAA0EA76EF8
:10006A00A68212000401226B010E236F1200000106
:10007A00756B65D90AE270D90800F5CF76F00001F0
:10008A0057D976C0EFFF752BF4D7F86A1200F00E35
:10009A0004012217840EA66E0001756B50D90AE27C
:1000AA0053D90F0E000175150F0801E1D5DF0001C4
:1000BA00752BF4D71200940EA66E0001756B3FD90A
:1000CA0011E27551006E016A060ED89000360136AB
:1000DA00E804FBE1026A01BE02681BD9BDDF000128
:1000EA00752BEDD7F86A1200A66A0001756B27D93D
:1000FA000BE20401225100017525A96EA68018D9C8
:10010A00A8CFEFFF752BF3D712000001756B17D933
:10011A0010E20401225100017525A96E09D9EF5098
:10012A00A86E040EA66E98DFA6B2FED70001752B44
:10013A00EED71200C40EA66E0001756B00D905E257
:10014A0003D98ADF0001752BF9D7F86A1200A0D803
:10015A00060E00017A5D03E36D50020B01E097D0B1
:10016A000001770511E104010CBF0DD00401400E16
:10017A00096F400E040108170401087D880E040166
:10018A0008130001776B83D0040108BF80D00001F7
:10019A00756B04012051320A45E0CD0A34E0F80AB1
:1001AA002DE0020A26E0010A1FE0070A18E0010A08
:1001BA0011E0030A0AE0070A08E0060A01E056D03D
:1001CA0051DF0001040E756F52D051DF050E000198
:1001DA0075274DD05CDF0001010E756F48D06BDFCB
:1001EA000001010E756F43D07FDF050E00017527F0
:1001FA003ED08BDF0001010E756F39D09BDF000105
:10020A00010E756F34D06D960001786B796B000121
:10021A007807000E795B00017851791101E0F7D770
:10022A00FF0025D0030E0401215D0DE104012251D6
:10023A00010BF36EF346F346FB0E8C14F310000029
:10024A000001010E756F040E0401215D0EE1040127
:10025A002251010BF36EF346F346F346F70E8C1464
:10026A00F31000000001010E756F01D000D00001EB
:10027A00010E776F000175510AE075C00DF4400E4A
:10028A0004010C1704010C7D880E04010C131200E2
:10029A0000017E517F1104E1200E7E6F4E0E7F6FAA
:1002AA007E07000E7F5B6DA208D07E517F1130E180
:1002BA0000008C50010B13E128D000017A5102E1B1
:1002CA00000023D07A0502E1000009D0020E7A5D0F
:1002DA0002E100001AD0030E7A5D03E1000000007B
:1002EA001200050E7A5D06E100017E517F1110E1D0
:1002FA0000000BD0060E7A5D0BE100017E517F11E2
:10030A0007E100000000010B02E0000012000000FB
:10031A001200040122510024F36E23510120F46ECD
:10032A0024510220F86EF4CFF7FFF3CFF6FF120044
:10033A007551EA6A250FE96E040EEA2212000401D9
:10034A0021510001755D1200F3DFEFCF03F004D8ED
:10035A0003C0F5FF0C00120075C000F0016A026AC2
:10036A008EEF01F06C5002E0000E01D0010E000980
:10037A000BE0040100513C0BE842E8420D0802E19F
:10038A00D2EF01F0DBEF01F06C5002E0000E01D079
:10039A00010E040901E019D812000001606B616BBB
:1003AA00666B676BA6EC02F05DEF02F0020E0001CD
:1003BA00605D09E15CD8040100BD02D0C80E01D01D
:1003CA00880E006F120096EF02F0040E00017A5DAB
:1003DA0009E112C46EFF6E50000802E2050E01D058
:1003EA00030E7A6F0001600509E10AD8040104BD11
:1003FA0002D0C80E01D0880E046F120096EF02F0E8
:10040A000001080E665D000E675903E266C069F0D6
:10041A0002D0080E696F69C005F46951006E016A5D
:10042A000050665F0150675B180E646F040E656FBB
:10043A0069511CE000017BA307D062C0F6FF63C0CC
:10044A00F7FF0800F55005D062C0E9FF63C0EAFF74
:10045A00EF5064C0E9FF65C0EAFFEF6E0001622B4E
:10046A00000E6323642B65236907E2D7120001C4D7
:10047A006AF000016A516625666F000E6721676F90
:10048A00180E626F040E636F6A5111E062C0E9FFD1
:10049A0063C0EAFFEF5064C0E9FF65C0EAFFEF6E90
:1004AA00642B000E6523622B63236A07EDD71200C3
:1004BA000001615105E13DD8840E006F04011DD091
:1004CA00040110AF1CD0000166510401165D000141
:1004DA0067510401175904E216C466F017C467F09D
:1004EA008FDF0001010E606F24D8800E006F0401B7
:1004FA00180E066F040E076FC80E046F10D00001A5
:10050A00020E606F0401056BC80E046F0401080E29
:10051A00016F180E026F040E036FC80E006F6D98FC
:10052A0012000001606B05D8880E006F0401046B8D
:10053A0012000401080E016F100E026F040E036F01
:10054A00120004011051600BE842E842E842E84216
:10055A00E842000901E012001151080A39E0010AD3
:10056A0035E00F0A0AE0030A01E012000001010E59
:10057A00616F0001040E7A6F12000001010E616FB3
:10058A000401130507E10001600E626F070E636F35
:10059A00120E13D0020E135D07E10001720E626F94
:1005AA00070E636F200E09D0030E135D0AE10001E6
:1005BA00920E626F070E636F040E0001666F676B1F
:1005CA0002D00001616B00017B831200FBEF02F095
:1005DA000001010E616F00017C0E626F000E636FF5
:1005EA0000017B930001010E666F12000001010EEB
:1005FA00616F12C47CF00401125104E10001050E7E
:10060A007A6F12000001060E7A6F1CEF00F0080ED6
:10061A006D6E6DBAFED7686A110E696E0001020E20
:10062A007A6F12006850040B06E06950040B03E06D
:10063A006D92699468946850010B04E06950010B4B
:10064A0001E027D86850100B09E06950100B06E04A
:10065A00698468986D82A08A0300A19A6850200B69
:10066A0009E06950200B06E070A003D096EC02F076
:10067A007090689A030E00017A5D01E209D0685011
:10068A00080B06E06950080B03E0B7EC01F0689626
:10069A001200686A7B0E696E6E6A160E706E68A624
:1006AA0002D06896FCD76D9896EC02F000017C6B3C
:1006BA000001030E7A6F12002A0EF66E000EF76E14
:1006CA00000EF86E00010900F550706F0900F55030
:1006DA00716F03E1706701D03DD00900F5506B6F6F
:1006EA000900F5506C6F0900F5506D6F090009009B
:1006FA00F550E96E0900F550EA6E09000900090093
:10070A00F5506E6F0900F5506F6F09000900F6CFBA
:10071A0072F0F7CF73F0F8CF74F06BC0F6FF6CC0CD
:10072A00F7FF6DC0F8FF00016E5302E16F5307E057
:10073A000900F550EE6E6E07F8E26F07F9D772C03E
:10074A00F6FF73C0F7FF74C0F8FF00017007000ED0
:10075A00715BBFD712001201000200000008D80422
:10076A000B000000000000010902200001010080C6
:10077A0032090400000200000000070501024000DF
:10078A00000705810240000004030904C1CF80F07C
:10079A000F0EC11281A804D080C0C1FF00EF04F07F
:1007AA000000000000000000140E6F6E0CEC03F055
:1007BA0017EC03F0ACEC00F0FBD7120013EE00F0DC
:1007CA0023EE00F0F86A059C61EC03F0CBEC03F031
:1007DA00FDD712000000FFFFFFFFFFFFFFFFFFFF33
:10080000BEEF0CF01200FFFF1200FFFFFFFFFFFF23
:100818001200FFFFFFFFFFFFFFFFFFFFFFFFFFFFCC
:10082A0001009E1900000801000002000000F00EFD
:10083A008C1695169388938A8150100B01E0010E4D
:10084A000001606F8150200B01E0010E616F99EC8D
:10085A0009F09280010EC26E3C0EC06EC08E37D86F
:10086A000001646B970ED56E12002AD9060E00019C
:10087A00F95D03E36D50020B01E028D031D8000185
:10088A00640524E1F2A422D0F294480ED76EE50E54
:10089A00D66EACEC09F0000919E00001A551E96E29
:1008AA00EA6AD890E936EA36A70EE926000EEA2265
:1008BA00E3C0EEFFE4C0EDFF1E0EA65D01E2A62B2B
:1008CA001D0EA55D02E1A56B01D0A52B120000014A
:1008DA00A56BA66B1200C282C2B2FED700D012006C
:1008EA00D9CFE6FFE1CFD9FFE652400EE66E650E9C
:1008FA00E66E000EE66E6FEC0BF0E552E552E5523D
:10090A00000901E1D8D00001626B00016551FF0ABC
:10091A0001E1BDD0C80A01E1B1D0010A76E0030ABB
:10092A006CE0010A5EE0070A55E0010A2EE0030ABC
:10093A000CE0310A01E0ADD00001676B0001010E45
:10094A00686F0001040E626FA5D00001010E626F8C
:10095A000001665103E18C948C9616D0000166055D
:10096A0003E18C948C8610D0020E0001665D03E1CF
:10097A008C848C9609D0030E0001665D03E18C8499
:10098A008C8602D00001626B85D0030E0001665D81
:10099A000EE100016751010BF36EF346F346FB0EBD
:1009AA008C14F3108C6E0001010E626F12D0040ECB
:1009BA000001665D0EE100016751010BF36EF3461B
:1009CA00F346F346F70E8C14F3108C6E0001010EF9
:1009DA00626F60D00001646B7ADF0001010E626F02
:1009EA0059D0ACEC09F0000907E0E3C066F0E4C0B6
:1009FA0067F00001030E626F4DD00001010E646FB3
:100A0A0066DF0001010E626F45D00001A651E8249D
:100A1A00020F0001626F0001A651E8240001666F0F
:100A2A00A6C0DFFFDF50000827E20001A55104E15C
:100A3A0000011D0EA56F02D00001A5070001A551F6
:100A4A00E96EEA6AD890E936EA36A70EE926000E78
:100A5A00EA22EECF10F0EFCF11F0EA6ADF34FE0B94
:100A6A00EA36E96E650EE926000EEA2210C0EEFFAC
:100A7A0011C0EDFFDF06D6D72ADF0CD02CDFC3CF9B
:100A8A0066F0C4CF67F00001030E626F03D0FF0067
:100A9A0001D000D0000162510EE004010CBF0BD05E
:100AAA0062C0E6FF650EE66E000EE66E35EC0BF0F0
:100ABA00E552E552E552E552E552E7CFD9FF120079
:100ACA0001010851091104E1100E086F270E096F80
:100ADA000807000E095B6DA20BD00851091107E146
:100AEA008C708C50010B02E08C8201D08C9230D039
:100AFA000001F95104E18C908C925ED829D0F90555
:100B0A0003E18C808C8224D0020EF95D03E18C8093
:100B1A008C921ED0030EF95D03E18C908C8218D062
:100B2A00050EF95D07E101010851091102E18C7016
:100B3A008C920ED0060EF95D0BE1010108510911E4
:100B4A0007E18C708C50010B02E08C9201D08C82F0
:100B5A0012008150100B01E0010E0001605D09E0F6
:100B6A008150100B01E0010E606F81B802D0010EB6
:100B7A0002D0000E00D012008150200B01E0010EBD
:100B8A000001615D09E08150200B01E0010E616FF7
:100B9A0081BA02D0010E02D0000E00D01200D9CFC5
:100BAA00E6FFE1CFD9FFACA2FED7FE0EDB50AD6E59
:100BBA00E552E7CFD9FF1200D9CFE6FFE1CFD9FF3F
:100BCA00E652C7DF000901E1D3D08C80C2DF0009F9
:100BDA0001E1FCD78C908C82CFDF000901E1FCD7C0
:100BEA008C928C84C9DF000901E1FCD78C948C8635
:100BFA00C3DF000901E1FCD78C96C66A948E949CE7
:100C0A00710EAF6E020EB06E240EAC6E900EAB6E0D
:100C1A00080EB86EAE50DF6EAE50DF6EADDF000963
:100C2A0001E1FCD7520EE66EBADFE552530EE66ECC
:100C3A00B6DFE5522D0EE66EB2DFE552320EE66EF3
:100C4A00AEDFE552330EE66EAADFE552320EE66EED
:100C5A00A6DFE552200EE66EA2DFE552540EE66EDE
:100C6A009EDFE552580EE66E9ADFE552200EE66EDA
:100C7A0096DFE552540EE66E92DFE552650EE66E99
:100C8A008EDFE552730EE66E8ADFE552740EE66E6B
:100C9A0086DFE552200EE66E82DFE5524F0EE66EE3
:100CAA007EDFE5524B0EE66E7ADFE5522C0EE66EDB
:100CBA0076DFE552200EE66E72DFE552500EE66EE2
:100CCA006EDFE552720EE66E6ADFE552650EE66E7B
:100CDA0066DFE552730EE66E62DFE552730EE66E6C
:100CEA005EDFE552200EE66E5ADFE552220EE66E10
:100CFA0056DFE552720EE66E52DFE552220EE66EBE
:100D0A004EDFE5522C0EE66E4ADFE5529EAAFED76A
:100D1A00720EAE5C2CE1200EE66E41DFE552520EF9
:100D2A00E66E3DDFE552580EE66E39DFE552200EDB
:100D3A00E66E35DFE552540EE66E31DFE552650E9A
:100D4A00E66E2DDFE552730EE66E29DFE552740E6C
:100D5A00E66E25DFE552200EE66E21DFE5524F0EE4
:100D6A00E66E1DDFE5524B0EE66E19DFE5525FDDDA
:100D7A00E552E552E7CFD9FF120004011851600B82
:100D8A00E842E842E842E842E842000901E055D078
:100D9A001951070A51E00B0A4FE0070A40E0010A1D
:100DAA002CE00B0A28E0020A26E0030A22E0080ADD
:100DBA0012E0010A0EE00F0A0AE0030A01E03CD041
:100DCA000101010E016F0001040EF96F36D036D809
:100DDA0034D090D832D00101010E016F0101FB0E0F
:100DEA00026F000E036F0001FA930101010E066FF4
:100DFA0024D0A8D822D0F6D820D00101010E016F44
:100E0A0004011C510101026F036BFC0E0227000E44
:100E1A0003230001FA930101010E066F0ED00101AE
:100E2A00010E016F04011C51EA6AFC0FE96E000E03
:100E3A00EA221AC4EFFF01D000D01200800E04018A
:100E4A00185D57E11B51030A34E0010A10E0030A56
:100E5A0001E04DD00101010E016F01015E0E026F2A
:100E6A00170E036F120E0101066F076B40D00101C6
:100E7A00010E016F04011A51F66EF76AD890F63620
:100E8A00F7360C0EF626180EF7220900F5CF02F1F6
:100E9A000A00F5CF03F1020E0101F76A0225F66E88
:100EAA000351F7220900F5CF06F10A00F5CF07F141
:100EBA001ED00101010E016F04011A51F66EF76A84
:100ECA00D890F636F736100EF626180EF7220900D5
:100EDA00F5CF02F10A00F5CF03F102C1F6FF03C113
:100EEA00F7FF0800F5500101066F076B00D00001FB
:100EFA00FA8312000101010E016F0F0EE66E710EE8
:100F0A00E66E0F0EE66E0BEC0BF0E552E552E5527B
:100F1A00010EE66EFC0EE66E000EE66E0BEC0BF0B2
:100F2A00E552E552E5521AC4FBF004011A5104E1F4
:100F3A000001050EF96F05D00001060EF96F20ECCD
:100F4A000BF012000401206B216B040118511F0BD6
:100F5A00020A16E0030A10E0010A01E035D0010195
:100F6A00010E016F80A402D0040120810001FAA1C0
:100F7A0002D00401208328D00101010E016F24D080
:100F8A000101010E016F04011C510F0B080DF350F2
:100F9A00116A000F106E040E11221C51800B01E021
:100FAA00010E040DF35001011024046F000E1120EC
:100FBA00056F04C1E9FF05C1EAFFEF50040B03E026
:100FCA000401010E206F00D0010101050AE10101AF
:100FDA00200E026F040E036F0001FA930101020E44
:100FEA00066F120004011A0510E118511F0B0009BF
:100FFA000CE10101010E016F030E0401195D03E109
:10100A000001FA8102D00001FA9104011A513AE171
:10101A0018511F0B020836E11C510F0B000932E070
:10102A000101010E016F04011C510F0B080DF35051
:10103A00116A000F106E040E11221C51800B01E080
:10104A00010E040DF35001011024046F000E11204B
:10105A00056F030E0401195D07E1840E04C1E9FF5F
:10106A0005C1EAFFEF6E0ED01CAF06D004C1E9FF3E
:10107A0005C1EAFFEF6A06D0880E04C1E9FF05C17F
:10108A00EAFFEF6E12006C5002E0000E01D0010E72
:10109A0000090BE0040100513C0BE842E8420D084C
:1010AA0002E10CD801D01CD808D06C5002E0000E26
:1010BA0001D0010E040901E023D81200D9CFE6FFBE
:1010CA00E1CFD9FFE6520101006B016B066B076B9A
:1010DA00C2EC06F0D5D8E552E552E7CFD9FF1200A7
:1010EA00020E0101005D0AE192D8040100BD03D09D
:1010FA00C80E006F02D0880E006F01D007D9120007
:10110A00040E0001F95D0AE11AC46EFF6E50000870
:10111A0003E2050EF96F02D0030EF96F0101000513
:10112A000AE10BD8040104BD03D0C80E046F02D033
:10113A00880E046F01D0EAD81200D9CFE6FFE1CFBA
:10114A00D9FF020EE1260101080E065D000E0759BD
:10115A0005E206C1DEFF07C1DDFF03D0080EDE6E21
:10116A00DD6A040104930491010EDB500413DFCFFE
:10117A0005F4000EDB500101065F010EDB50075B30
:10118A00200E046F040E056F0001FAA31ED0D9CFFA
:10119A00E9FFDACFEAFFEE50ED1016E002C1F6FFE2
:1011AA0003C1F7FF0800F55004C1E9FF05C1EAFFD2
:1011BA00EF6E0101042B000E0523022B0323DF0629
:1011CA00010E01E2DB06E3D71CD0D9CFE9FFDACF63
:1011DA00EAFFEE50ED1015E002C1E9FF03C1EAFF94
:1011EA00EF5004C1E9FF05C1EAFFEF6E0101042BCC
:1011FA00000E0523022B0323DF06010E01E2DB06A4
:10120A00E4D7D9CFE1FFE552E7CFD9FF1200D9CF12
:10121A00E6FFE1CFD9FF020EE126030E0401001515
:10122A00E76E010EE7CFDBFF01C4DFFFDE500101ED
:10123A000627DD500723200E026F040E036FD9CF55
:10124A00E9FFDACFEAFFEE50ED1014E002C1E9FF40
:10125A0003C1EAFFEF5004C1E9FF05C1EAFFEF6EDF
:10126A00042B000E0523022B0323DF06010E01E2E5
:10127A00DB06E5D7D9CFE1FFE552E7CFD9FF120068
:10128A00010101510CE10401080E016F180E026FF1
:10129A00040E036F840E006F0401046F35D004013D
:1012AA0018AF22D00101065104011E5D0101075148
:1012BA0004011F5904E21EC406F11FC407F13DDFF1
:1012CA000101010E006F0401080E016F180E026F72
:1012DA00040E036F800E006F0401200E066F040EC9
:1012EA00076FC80E046F10D00101020E006F0401CF
:1012FA00056BC80E046F0401080E016F200E026F01
:10130A00040E036FC80E006F6D9812000101006B86
:10131A000401080E016F180E026F040E036F880E87
:10132A00006F0401046B12008A849394E66A030E28
:10133A00E66E020EE66E5AEC0CF0E552E552E55204
:10134A000001870EE36F0C0EE46FBDEF09F08A947B
:10135A00CAEC0CF00001E46FCAEC0CF00001E36F78
:10136A008A84E3B502D0000E02D0010E00D012002A
:10137A00D9CFE6FFE1CFD9FF030EE126E3C010F093
:10138A00E4C011F0D89011321032E804FBE110C029
:10139A00DEFF11C0DDFFD950010FE96EDACFEAFF97
:1013AA00EF50100B08E1010EDB9ADB9CDB9E00017B
:1013BA002B0EE56F16D0010EDB8ADB8CDB8E00016B
:1013CA002D0EE56FDECF10F0DDCF11F0FF0E101AF3
:1013DA00111A10C0DEFF11C0DDFFDF2A010E01E382
:1013EA00DB2ADECF10F0DDCF11F00A0E1102F3CFA7
:1013FA0011F01002F3CF10F0F4501126040ED89019
:10140A0011321032E804FBE110C0DEFF11C0DDFF2B
:10141A00040EF36E020EF3CFDBFFDB50000833E25B
:10142A00DECF10F0DDCF11F00A0E0B6E0C6A10C081
:10143A0006F011C007F0A8EC0CF002C010F003C0CF
:10144A0011F00F0E10143009E66E020EDB50EA6A34
:10145A00E50FE96E000EEA22E552E750EF6ED9CFAA
:10146A00E9FFDACFEAFF0A0E0B6E0C6AEECF06F03E
:10147A00EDCF07F0A8EC0CF006C0EEFF07C0EDFFB9
:10148A00020EDB06CAD7300E0001E65D07E1200E28
:10149A00E66F300EE75D02E1200EE76FE9C0EAF081
:1014AA002E0EE96FF80EEB6F430EEC6F0D0EED6F1B
:1014BA00EE6BD9CFE1FFE552E7CFD9FF120080A248
:1014CA0003D06DA60FD802D06DB613D80001F90566
:1014DA0008E16DBA06D0686A696A69806988020E8D
:1014EA00F96F12006D6A696A6D860001010EF96F63
:1014FA0012006D6A696A0001F96B12007EEF0AF048
:10150A000001F95101E13AD06850040B04E0695036
:10151A00040B01E038D86DB231D06850010B04E0F9
:10152A006950010B01E050D86850100B04E0695073
:10153A00100B01E024D86850400B04E06950400BBE
:10154A0001E037D86850200B04E06950200B01E015
:10155A0032D86850020B04E06950020B01E032D81D
:10156A00030E0001F95D01E209D06850080B06E09C
:10157A006950080B03E048EC08F068961200698489
:10158A0068986D8212006D92699468941200000145
:10159A00FAA10ED0F8DF6D840001080EFD6F070E68
:1015AA00FE6FFD07000EFE5BFD51FE11FAE16D9420
:1015BA001200689C120070A003D08BEC09F07090A6
:1015CA00689A1200689212006A6A686A9F0E6B6EC5
:1015DA007B0E696E6E6A0F0EE66E710EE66E0F0E68
:1015EA00E66E14D8E552E552E552160E706E68A6FC
:1015FA0002D06896FCD76D988BEC09F00001FA913D
:10160A000001FB6B0001030EF96F1200D9CFE6FF50
:10161A00E1CFD9FFFD0EDBCFE9FFFE0EDBCFEAFFFC
:10162A00FC0EDB5004E0EE6AFC0EDB06F9D7E5524D
:10163A00E7CFD9FF12000001FF6B1E0E716E040185
:10164A00400E096F280E0A6F040E0B6F880E086F82
:10165A000401680E0E6F040E0F6F400E0C6F12001D
:10166A00D9CFE6FFE1CFD9FFE652FC0EDB504008A6
:10167A0005E2400EF36EFC0EF3CFDBFFDF6AFC0ED1
:10168A00DB50DF5C19E2DF50E76EFD0EDBCFE9FFCE
:10169A00FE0EDBCFEAFFE750E926000EEA22EF5002
:1016AA00E66EDF50EA6A680FE96E040EEA22E55236
:1016BA00E750EF6EDF2AE3D7FC0EDBCF0DF4400EC6
:1016CA0004010C170C7D880E0C13E552E552E7CF86
:1016DA00D9FF1200D9CFE6FFE1CFD9FF0001FF6B96
:1016EA00040108BF30D0FC0EDBCF10F00951D880BE
:1016FA00105403E2FC0E09C4DBFF0001FF6BFC0E71
:10170A00DB50FF5D19E2FF51EA6A280FE96E040E09
:10171A00EA22EF50E66EFF51E76EFD0EDBCFE9FFDE
:10172A00FE0EDBCFEAFFE750E926000EEA22E55279
:10173A00E750EF6EFF2BE3D70401400E096F08173D
:10174A00087D880E08130001FF5100D0E552E7CF4B
:10175A00D9FF12001201000200000008D8040C0090
:10176A000000010200010902200001010080320983
:10177A0004000002000000000705010340002007E2
:10178A000581034000200403090434034D00690065
:10179A00630072006F006300680069007000200037
:1017AA0054006500630068006E006F006C006F00F3
:1017BA0067007900200049006E0063002E00440390
:1017CA00500049004300440045004D0020004600F7
:1017DA0053002000550053004200200044006500D9
:1017EA006D006F00200042006F006100720064000B
:1017FA002000280043002900200032003000300079
:10180A0034007017701790179417C8172A0EF66EBF
:10181A00080EF76E000EF86E00010900F550F46F1D
:10182A000900F550F56F03E1F46701D03DD00900D6
:10183A00F550EF6F0900F550F06F0900F550F16FA0
:10184A0009000900F550E96E0900F550EA6E090031
:10185A0009000900F550F26F0900F550F36F09000D
:10186A000900F6CFF6F0F7CFF7F0F8CFF8F0EFC0AF
:10187A00F6FFF0C0F7FFF1C0F8FF0001F25302E1F2
:10188A00F35307E00900F550EE6EF207F8E2F307AA
:10189A00F9D7F6C0F6FFF7C0F7FFF8C0F8FF000166
:1018AA00F407000EF55BBFD71200D9CFE6FFDACFF7
:1018BA00E6FFE1CFD9FFE2CFDAFF3F0EC716C66ACD
:1018CA00FD0EDB50C612FB0EDB50C712FC0EDB50BE
:1018DA00030A09E0010A04E0020A06E1C78C04D0FF
:1018EA00C78CC68801D0C688FD0EDB50050A03E006
:1018FA00010A04E1928A9382C79E01D09392949E30
:10190A009380C68AE552E5CFDAFFE7CFD9FF120006
:10191A0005D812D83AEC04F0FCD712000F0EC11207
:10192A0092829284140E6F6E0001F96B0001FA6BB9
:10193A000001FB6B1CEF04F064EC0AF06FBE02D0EE
:10194A0085EC0AF01200036A026A100EE76ED8905C
:10195A0006360736023603360B50025C0C50035823
:10196A0005E30B50025E0C50035A062AE72EF0D705
:10197A00120013EE00F023EE00F0F86A0F9C0BEC55
:10198A000CF08DEC0CF0FDD71200C96AC7A0FED787
:10199A00C95012000000FFFFFFFFFFFFFFFFFFFF1C
:020000040020DA
:020000040030CA
:0E000000240E3F1E008181000FC00FA00F4094
:0200000400F00A
:00000001FF
